:1000000000308A00842900000A108A100A11820731
:1000100028340C34013406340A108A100A1182077D
:1000200047346D34653474347234203430342E34B3
:1000300031342E34323420344234653474346134F3
:1000400000340A108A100A1182074B3461346B3471
:100050006C3469346B3440346D346C3461346234E4
:100060002E3463347A3400340A108A100A1182075D
:1000700043346C34693462347234613474346934B6
:100080006F346E342E342E342E3400340A108A101D
:100090000A1182072A34003436308400000803191C
:1000A00060280130A100A001A00B5428A10B532807
:1000B0004A30A000A00B5A2800000000800B5128F5
:1000C000003407080F39BD003C0EA000F030A00539
:1000D0002008F0393D04870006148316061000003E
:1000E000831206108316061083120034BA08031D0B
:1000F0007B2886107C288614831686108312BB0EFC
:100100003B08BC006120BB0E3B08BC0061200D30E9
:10011000A000A00B892800341430B6004C200F300A
:1001200083168705831286108316861083120610A5
:10013000831606108312AB012B08023C031CA8286F
:100140000230B6004C200330BC006120AB0A9C2872
:100150000D30A000A00BAA280230BC0061200D3099
:10016000A000A00BB128AB012B08023C031CC42843
:100170002B080420AC00BA012C08BB00762002300A
:10018000B6004C20AB0AB4288A11BD2901303602D2
:10019000B8003708023C031DCF284030B8073808A4
:1001A0008038B900BA013908BB0076200034350820
:1001B0000C3A0319E528063A0319ED28073A031902
:1001C000F328053A0319F828FD28BA010130BB00CD
:1001D00076200230B6004C2009290130B6000230EA
:1001E000B700C62009290130B600B700C62009298A
:1001F000BA011030BB007620092935081F3C031CCA
:1002000003290730B5050130BA003508BB00762058
:10021000092900340C30B500D72000340408B4009C
:10022000AE1F1A29B417341EB40AAD09AE09AD0ABF
:100230000319AE0A2E0EF038B000B007E23EB1004E
:10024000323EB3002E080F39B107B107B307E93EBC
:10025000B200B207B2072D0E0F39B207B307B20DC5
:10026000B30DB309B30D2D080F39B307B00D073027
:10027000AF000A30B307B203031C3A29B207B10337
:10028000031C3E29B107B003031C4229B007AF038A
:10029000031C46292F3084000730340534138403AF
:1002A0003405031D5A29341A840A341A5A29203075
:1002B000A00077298407333004020319341700089B
:1002C000A000031D6B29341B6B29341A7F29B41934
:1002D0006B2920307629B41F73292D30A0008403A8
:1002E0003413B4137729B41534123030A007AE019B
:1002F0000408AD002008B500D7202D088400840A2A
:10030000341F5B298A11472A84011F308305831615
:100310001F149F141F159F11FF308312A500831611
:100320001F109F101F119F1183121F139F138316FD
:100330009F1783121F149412A51225088316870095
:10034000831225162508831687008312A511250818
:1003500083168700003083129400831694000108EE
:10036000C73908388100831290010030A100920043
:1003700000308316920083128C286430B6004C2023
:100380000830A1001F08C73921049F000130B600C2
:10039000B700C620AB012B080C2000380319D42964
:1003A000AB0AB500D720CB290130B6000230B70028
:1003B000C620AB012B08212000380319E329AB0A22
:1003C000B500D720DA290230AB00FA30B6004C2055
:1003D000AB0BE5290A210130B600B700C620AB01FE
:1003E0002B08342000380319F929AB0AB500D720AF
:1003F000F029A701A601A90129087F3C031C102AA6
:100400000A30B6004C201F151F19042A83161E0837
:100410008312A6070318A70A1E08A707A90AFC2922
:10042000A70CA60CA70CA60CA70CA60CA70CA60C38
:10043000A70CA60CA70CA60CA70CA60C0130A705B0
:100440001F151F19212A83161E088312A800323097
:10045000B6004C200A210630B6000130B700C62095
:10046000A3012808A000A81BA3032602AB002708AD
:10047000AC002308031C230FAC022030B500D720AA
:100480000B3084002C08AE002B08AD000E29203064
:10049000B500D720A3012808A000A01BA303A1003A
:1004A000A71F552AA31F612A572AA31B782A2708AA
:1004B0002302031C782A031D612A26082102031C3B
:1004C000782AA3012808A81BA303A100260821025B
:1004D000A0002708031C270FA3022008AA002A0E49
:1004E000A000A00C0730A0052008083EAA008C2A16
:1004F000A3012808A81BA3032602A0002308031CAD
:10050000230F842A2708852A2702A3002008AA008F
:10051000AA0EAA0C0730AA052A08B6000230B700B6
:10052000C620AB012B084620003803199B2AAB0AD2
:0A053000B500D720922A202A6300AC
:02400E00393F38
:00000001FF
